:020000040000FA
:020000001028C6
:080008001F2A8207C034F934FD
:10001000A434B034993492348234F8348034903437
:1000200003138312850107309F008316203085005B
:10003000003086000A308E00883081000C10831258
:100040008B120130900005170B178B17C601CA01E0
:10005000C801C501D601F721B32183161F308600E0
:10006000831206081F391F3AC400831686018312C3
:10007000441D3E280130C806A421F5214518592801
:10008000441C2D281321C419E9280513C820CB01CD
:10009000CC01CD01CE01CF014614C7010530CA0005
:1000A0004514483081001330C0008830C1008B16E1
:1000B00079284418B028C41C602820308B06642896
:1000C000C41D67280630CA00A421F5212D284A083E
:1000D00003196C2803303E21461C2D284A08031DB5
:1000E000CA034F08031D79284E08031D79280530DF
:1000F000CA004F08031D8B280310C60D4E08031DB0
:100100008B28C60DD320B620461A8B284D08031D18
:100110008B280310C60D4708031994288B21FA3049
:10012000E221C70B8E28AE28C60C031C9A28481C57
:100130007D21AE28C60C031C9F288421AE28C60C46
:10014000031CA4289921AE28C60C031CAB289721B8
:100150004C08C700AE288F21F5218F21C6012D281C
:100160008B12C501DF308500AF212D28D00803197F
:10017000BF285408D1020318BA28D003B72854085E
:10018000D102031CC728031DC0281030C600080078
:100190005308D40052080319D228D5000A30D407D6
:1001A000D50BCE280800D0014D08D1004C0803190A
:1001B000DE28D5000A30D107D50BDA284B08031901
:1001C000E828D5003C30D1070318D00AD50BE22827
:1001D0000800A421F521F521561403303E21831691
:1001E0001F308600831206081F391F3AC400831689
:1001F00086018312C418052144190C21C41DED2861
:100200002521A421F521D6012D28D20A0A30520237
:100210000318D201F5210800D30A0A30530203184B
:10022000D301F5210800831626309B00831252303B
:1002300084000230D70083161C141A089B0A83120C
:100240008000840AD70B1B290800831626309B00E8
:100250008312523084000230D700000883169A00BF
:100260001C1555309D00AA309D009C149C18362901
:100270009B0A8312840AD70B2D290800C900FF307E
:1002800086000514F730561848294B0805207F3999
:1002900086000512DD21FF30860005164C08561831
:1002A0005208052086008511DD21FF308600851566
:1002B0004D08561853080520561C7F398600051135
:1002C000DD21FF3086000515F730561869294E08E4
:1002D000052086008510DD21FF3086008514F7306B
:1002E000561874294F08052086000510DD21C90B1A
:1002F0003F29FF30860005140800FB30C20004309F
:10030000C3006430D5210800FC30C2004430C30073
:100310006430D52108007D21EF21842108008B2144
:10032000EF218B21EF218B21EF218B2108009921D7
:10033000EF218421EF2184210800F830C2008930A8
:10034000C3006430D52108009D21EF219D210800C4
:10035000F830C2008930C300FA30D52108009D2151
:10036000F321A8210800F830C2008930C300C8304A
:10037000D521F121FA30C2001330C300C830D52195
:10038000F121FB30C2000430C300C830D521F12177
:10039000FC30C2004430C300C830D521FC30C2005C
:1003A0004430C300C830D521080083160C148312D2
:1003B000E22183160C10831208006430DC00DC0B91
:1003C000DF290800DB006E30DA00E629E729E8299A
:1003D000DA0BE529EB29EC29DB0BE32908001E30B9
:1003E000E2293230E2296430E229C830E229FD21D5
:1003F0000E22FD210E22FD2108000530D9007F309C
:1004000086000130D800580985000310D80DF3216B
:10041000DF308500F121D90B032A08000530D9000F
:100420007F3086001030D800580985000310D80CA2
:10043000F321DF308500F121D90B142A0800F000E8
:100440000308F10083120B19282A0C185A2A612A72
:100450000B11483081000130C1020319332A0318FF
:10046000612AC002612AC008031D612A1330C0003E
:100470008830C1004614CF0A0A304F02031C612A9B
:10048000CF01CE0A06304E02031C612ACE01CD0AEE
:100490000A304D02031C612ACD01CC0A06304C0201
:1004A000031C612ACC01CB0A0A304B02031C612ACF
:1004B000CB01612A0C1042088F0043088E00803067
:0C04C000850671088300F00E700E090024
:02400E00103F61
:1042000043006F0070007900720069006700680069
:1042100074002000280043002900200032003000F4
:10422000310036002D003200300031003700200010
:104230006200790020004D002E00590061006D00E1
:1042400061006D006F0074006F00FF00000000004F
:00000001FF
